:030000000219FDE5
:03000B000200AA46
:03002B000201656A
:03005B000202F8A6
:030073000202DEA8
:1000800002030406080C10182030406080040608A3
:100090000C10182030406080A0C000070F1F3F0DDB
:1000A0000D04050D050305030302C2AFC0D0C0E077
:1000B000206217E5256002E473E525F4F58A758B67
:1000C00000D262D0E0D0D0D2AF3285268AC262E5BB
:1000D00026F46035306803207210758B00D0E0D0B4
:1000E000D0D292D291D290D2AF32D292D291D2903B
:1000F000206E0C206609740AD5E0FDE57E429075FD
:100100008B00D0E0D0D0D2AF32758A00C28DD262DF
:1001100001FF01B9306805206602C29201B930685A
:1001200005206602C29101B9306805206602C290BE
:1001300001B9C29330680A2066077408D5E0FDC291
:100140009201B9C29430680A2066077408D5E0FDB0
:10015000C29101B9C29530680A2066077408D5E0DB
:10016000FDC29001B9C2AFC2AD53E6EFC0D0C0E04E
:10017000D2D3D2AFC2CEE52A6007207449152A2116
:10018000C67800790020742EE580307E01F430E4DA
:100190000278FF53DACF207E0343DA20307E034318
:1001A000DA10C2D8C271E580307E01F430E4027901
:1001B000FFC3E89970CB306103752A18207403756A
:1001C0002A18885FD27020740DE52B6004152B214E
:1001D000D643DA01C2D82070024134A85F20610200
:1001E000C2702074367982B70431C3E894F04003BA
:1001F00074F0F8E8C4540F28F87984B70302411B5F
:10020000C313C3138721200802C313200A06C3C8DF
:1002100098F8411B28F8500374FFF88822E52D5404
:10022000066011E533C313C31324062522F52250BB
:10023000037522FF7882B60459852224A824C3E5D9
:100240002495644002A864C3E895664002A86688C5
:1002500025E56970024185C3E8AA699A5003E8FA66
:10026000E4F9EAC333FBE56BF45B29400D256AF83A
:10027000E56A6002156A400B41850AC3E56A9A5037
:1002800002056A78FF8826C26EC3E52694F840020C
:10029000D26EC3E52594404002D26420CF0AD0E05C
:1002A000D0D043E610D2AD32C2CF053A7801E52A6C
:1002B0006005307402152AC3E55F9401400575623C
:1002C0000041D4756300756C00E5622401F562504D
:1002D000037562FFD0E0D0D043E610D2AD32C2AF9A
:1002E000C0D053E67FC260759100855694855795BE
:1002F000759104D0D0D2AF32C2AF53E6EFC2ADC0D9
:10030000D0C0E0C0F0D2D3D2AFA8FBA9FCC2D83095
:100310007102615F53DACF207E0343DA10307E032F
:1003200043DA20D271E580307E01F420E4026136A8
:1003300088278928A18C53DACF207E0343DA203026
:100340007E0343DA10C2D8C271307402A1787800FB
:10035000E580307E01F430E402A178885FA160532B
:10036000DACF207E0343DA20307E0343DA10C271F5
:10037000206102813853DACF207E0343DA10307EC9
:100380000343DA20C2D8D271885A895BC3E89558F2
:10039000F8E99559F97B007E087A00C3E8948CE966
:1003A00094005005755E00812A882178A2E6A82174
:1003B0006055C3E894C8E994005008E4D2E4FB7A9D
:1003C0000A8105C3E89468E994015008E4D2E3FB8C
:1003D0007A0F8105C3E894D0E994025008E4D2E290
:1003E000FB7A1E8105C3E894A0E994055008E4D285
:1003F000E1FB7A3C8105C3E89498E994085008E44D
:10040000D2E0FB7A787E00C3E8955CFCE9955DFD5F
:1004100030E70AECF42401FCEDF43400FD755E00D5
:10042000C3EC9AED9E5003755E01885C895D855A28
:1004300058855B597802A160C3E89527F8E99528AB
:10044000F9307C02A144307B02A144307A02A13D04
:10045000207502815BE9FDE8FC817AE9C313F9E8C4
:1004600013F8307902A13DE9C313F9E813F83078A5
:0F04700002A13DE9C313FDE813FC20612CC3EC8E
:10047F00941CED940240028191ED701EC3EC94C860
:10048F0050180529E52970021529C3E529940A504A
:10049F0002A178755F00D270A178E5296002152955
:1004AF007888E6F97400207F087896B90302789E61
:1004BF00E624FAFEE43400FFC3EC9EFCED9FFD92B0
:1004CF0008B90310A2085007207609D27681E330CD
:1004DF007602C276A2085016B9030DECF42401FC83
:1004EF00EDF43400FD0204FD78007900A144B90356
:1004FF0015EC33FCED33FDC3EC940AFCED9400FDD9
:10050F0050047C007D00C3EC94FFED94004006780E
:10051F00FF7900A144EC8575F0A4C5F0A2F733F87C
:10052F007900400302056078FF7900020560E9C396
:10053F0013F9E813F8307C0EE9600278FFC3E81373
:10054F0038F8E43400F9C3E894FFE99400400278E6
:10055F00FF885FD270206102A178741FF4552F4B72
:10056F00F52FC274EB7002D274752A1830740375AC
:10057F002A0A306102A18C20740353DAFE2074031F
:10058F00752B06D0F0D0E0D0D0D2AD43E610327943
:10059F00010205BC79030205BC790A0205BC791E6C
:1005AF000205BC79640205BC79C80205BC7817E462
:1005BF00D5E0FDD8FAD9F6227A147B780205E37AD2
:1005CF00107B8C0205E37A0D7BB40205E37A0B7B7B
:1005DF00C80205E37902B27DE4C294D5E0FDC29171
:1005EF00D5E0FDD291D5E0FDD294D5E0FDC292E5E4
:1005FF0076D5E0FDD2927496D5E0FDD9D9EAF8D53B
:10060F00E0FDD8FBDBCEC29422C37C007D0075F0E9
:10061F000005F0EA33FAEB33FB50F6EB13FBEA136A
:10062F00FAC3E9FFE8FEE89AF8E99BF95004EFF9FD
:10063F00EEF8B3EC33FCED33FDD5F0DFEDF9ECF86C
:10064F0022E889F08A20D2D4F8A9F07B0030F70B8A
:10065F007BFFF42401F8E9F43400F9E88520F0A4D5
:10066F00ADF0F8E98520F0A4AFF0FEED2EF974009F
:10067F003FFA7C04C3EA13FAE913F9E813F8DCF440
:10068F008BF030F70AE8F42401F8E9F43400F9E8C4
:10069F0089F0C2D4F8A9F0227882B60403020702C7
:1006AF00C3E55F940140030206CC852224E4F5459F
:1006BF00F546F547F548F549C26D0207027882E61F
:1006CF00FCD26DE522F523783879C7AA40AB41C338
:1006DF00EB13FBEA13FAEC146013C3EB13FBEA13EF
:1006EF00FAEC14146007C3EB13FBEA13FAD1188862
:1006FF0045894622C3E5459523F8E5469400F95010
:10070F000CC3E89480E994FF4016020733C3E894C2
:10071F007FE994005003020733787F790002073393
:10072F00788079FF884A894B22E54A2547F8E54BBF
:10073F003548F9854B20E4300701F43549FA30E7A5
:10074F0009C3EA94F04015020771C3EA940F5003EE
:10075F0002077178FF79FF7A0F020771780079002D
:10076F007AF0C3E5249564500AC374019524500BA5
:10077F0002078FE54B20E70E02078FE54B30E706A8
:10078F00884789488A492278A4E6FAC3E54A33F8AC
:10079F00E54B33F9D150E930E70BC3E89480E99486
:1007AF00FF4013E1C9C3E8947FE994005002E1C907
:1007BF00787F7900E1C9788079FFE820E715C3E5F4
:1007CF002398F84009C3E8940140030207F0780129
:1007DF000207F0E8F424012523F840030207F0781C
:1007EF00FF884C2278A5E6FAA848A949D150E930EC
:1007FF00E70CC3E89401E994FF4016020824C3E80C
:10080F0094FFE99400500302082478FF790002084E
:10081F0024780179FFE920E715C3E54C98F84009E2
:10082F00C3E89401400302084B780102084BE8F437
:10083F002401254CF8400302084B78FF88242278C6
:10084F00FFC26420693D206A12D264C3E541940A55
:10085F004009C3E52594405002C26479A1E76023A3
:0D086F00E541601F74FF8541F0848539F07C
:10087C00306A0375F005A4F8C5F0600278FFC3E890
:10088C0095675002A867886622C3E5409440E5410D
:10089C009401E56650031401A6046002F566220279
:1008AC0008AE2275E890227883E6FFE5E820ECF7A5
:1008BC00A8BDA9BE0573C3E57394084052757300B7
:1008CC00E9FA79A0E76044EA7007E574601B020856
:1008DC00E9C3E895746010E5745006600C140208C6
:1008EC00F50460F90208F5E574F574C39458401BDF
:1008FC007564C0C394044013756480C39404400BA6
:10090C00756440C39404400375640075BB0322E511
:10091C00642410500274FFF5647982B704022142FA
:10092C00C3A864E524985002A824C3E89566400245
:10093C00A86688258826E573B4070375BB10227456
:10094C003279A687F0A4C5F0A2F733F8C3E8956412
:10095C004002A86488228824882588268867227506
:10096C0040007541F022C2AF75C820A8CCA9CDAA11
:10097C003A30CF010A75C824D2AFAB3BAC3C883BB4
:10098C00893CC3E89BF8E99C206908F9306702416F
:10099C008721E4AD3D8A3DF9EA9DFA600478FF7940
:1009AC00FFAE3EAF3F8B3E8C3FC3EC9FFCC3E99C3C
:1009BC00F542A83BA93CC3E89EF8E99FF9C3E54181
:1009CC0013FBE54013FAE82AF540E93BF5415006E4
:1009DC007540FF7541FF412EAA40AB41AC40AD4183
:1009EC007E047F02C3EB940440021E1FC3EB9408E9
:1009FC0040021E1FC3ED13FDEC13FCDEF7C3EA9C93
:100A0C00FAEB9DFBEF6009C3E913F9E813F8DFF784
:100A1C00EA28FAEB39FB8A408B4150067BFF8B406E
:100A2C008B41C3EB94025002D2673069047F0341BF
:100A3C00597892E6FFC3E537948240110FC3E5372E
:100A4C0094A040010FC3EF940640027F057E05E59C
:100A5C0041C4540FF9E541C454F0F8E540C4540FB7
:100A6C0028F8C3E89EFAE99400FB4009C3EA940213
:100A7C00EB940050047A02E4FB41D3AA40AB41EB67
:100A8C00C4FEEAC4540F4EFCC3EA9CFAEB9400FB80
:100A9C00C3E813C313F8EA28FAEB3400FB8A408B43
:100AAC0041C3EB94024002C2677805EBC4FE7B00A5
:100ABC00EAC4540F4EFAC3EA98FA4005C3940250A4
:100ACC00027A027892E6FF30600241D38552568555
:100ADC005357D26043E680C3E49AF8E49BF930673D
:100AEC0002616DE8FAE9FBD3E913FDE813FC8852C7
:100AFC008953C3EF94036038EF20E00DE82CF8E93C
:100B0C003DF9ECFAEDFB020B28E828F8E939F9C3BA
:100B1C00E82402F8E93400F97AFE7BFFC3EF940372
:100B2C00400E8A548B55884E894F8C508D5161A143
:100B3C00885489558A4E8B4F8C508D51306920C307
:100B4C00E53394034019E542A2E713F8E555F42484
:100B5C000138400B20E7087554FFF42401F555616A
:100B6C00A1E8FAD3E813FC8852C3EF94036020EF9A
:100B7C0020E007E82CF8ECFA618DE8282402F87ADA
:100B8C00FEC3EF940340088A54884E8C5061A188B0
:100B9C00548A4E8C50E56BC3335002646BF56B304A
:100BAC00600261AB753402D26043E680E52D5406D9
:100BBC006026A840A941C3E913F9E813F8C2AF5362
:100BCC00E67F759100C3E498F594E499F5957591D9
:100BDC0004D26043E680D2AF22D265754400752002
:100BEC0000306B03752040020C04D265754400750F
:100BFC002040306B03752000D2AF7801206722E5CE
:100C0C002D54066002C265C3E54194054013780279
:100C1C009405400878039405400278063069027800
:100C2C000A206019E544601530690AC3E533940362
:100C3C004003D53406D2AFD26C81D671B3D2AF009B
:100C4C0000C2AF206726E541C3FB940F40027B0F27
:100C5C00EB240530730123306A02742820620123CF
:0E0C6C00F93069027982E58BC39940B50544E1
:100C7A00E59BF45440B5200281C030690A08C3E8F4
:100C8A00940A400108812D2065028104C26553E659
:100C9A007F7591003067107594007595FE75910403
:100CAA00D26043E6808104AE40AF41C3E49EF5942E
:100CBA00E49FF59581A7C3E533940250028104307D
:100CCA0065028104D80281D4812DC26C53E67F75F6
:100CDA009100855494855595759104854E56854F96
:100CEA0057D26043E680D2AFE52D54066008206AE9
:100CFA00020533020D10306C0D206B0A20650715B2
:100D0A0081158102158D22780030640530650278DC
:100D1A0001E53775F007A4F9E5F028F5F0E9A2F046
:100D2A0013A2F113A2F213F537C39478500375375F
:100D3A0078C3E53795384008D266D292D291D290DC
:100D4A00306002A14A855056855157D26043E680E9
:100D5A0022D2A0207D11C2AF754302C294D293D28F
:100D6A00AF759F10020F36C2AF754302C294D29577
:100D7A00D2AF759F10020F36C2A0307243207D2079
:100D8A00C2AF754303900143757E10D290C295306D
:100D9A006204C291A1A2D294D2AF759F20020F36EB
:100DAA00C2AF754303900143757E10D292C293304D
:100DBA006204C291A1C2D294D2AF759F00020F36CB
:100DCA00207D17C2AF75430390011ED29030620294
:100DDA00C291D2AF759F20020F36C2AF75430390FE
:100DEA00011ED292306202C291D2AF759F00020FE9
:100DFA0036D2A0207D11C2AF754304C293D295D2D8
:100E0A00AF759F00020F36C2AF754304C295D293E5
:100E1A00D2AF759F20020F36C2A0307243207D20C8
:100E2A00C2AF754305900132757E08D291C29430E3
:100E3A006204C292C142D293D2AF759F10020F369A
:100E4A00C2AF754305900154757E20D291C2943089
:100E5A006204C290C162D295D2AF759F10020F365A
:100E6A00207D17C2AF754305900114D291306202FA
:100E7A00C292D2AF759F10020F36C2AF754305906A
:100E8A000128D2913062EBC290D2AF759F10020F47
:100E9A0036D2A0207D11C2AF754306C295D294D234
:100EAA00AF759F20020F36C2AF754306C293D29424
:100EBA00D2AF759F00020F36C2A0307242207D2049
:100ECA00C2AF754301900154757E20D292C293300D
:100EDA006204C290C1E2D295D2AF759F00020F366A
:100EEA00C2AF754301900132757E08D290C2953027
:100EFA006204C292E102D293D2AF759F20E13620FA
:100F0A007D16C2AF754301900128D292306202C2A7
:100F1A0090D2AF759F00E136C2AF754301900114BC
:100F2A00D290306202C292D2AF759F20C2662290DE
:100F3A000112757E00D292D291D290C293C294C20B
:100F4A0095C26222788076090876090876040876BE
:100F5A00FF0876030876FF08760A08760308760102
:100F6A00087601788C76010876FF0876FF0876FF06
:100F7A000876FF0876FF0876030876FF0876FF08EA
:100F8A0076FF0876250876D00876280876500876FF
:100F9A00040876FF08760208760008767A0876FF53
:100FAA00087601087601087600087603227887E633
:100FBA00FFC272BF0302D2727888E6C39403600844
:100FCA00C27DE630E102D27DC27E7889E630E10256
:100FDA00D27EC3EF94026008758E01D273020FEFBE
:100FEA00758E00C273227880E6149000809378A4EC
:100FFA00F67881E6149000809378A5F67886E61450
:10100A0090008D9378A6F6789CE67538FF75390CB2
:10101A00B402067538A075390AB4030675388275A4
:10102A00390578A3E61490009A93F569120F3922CC
:10103A00227896E6FA7897E6FB7888E6B40305C341
:10104A00EB940EFB307F047A007BFFC3EB9AFCC360
:10105A00948250027C827575000575EC8575F0A442
:0F106A00C3E5F0947D40F222D27F113B1205AD19
:101079007A007B007C101205A3E55F2AFA74003B15
:10108900FBDCF37C04C3EB13FBEA13FADCF7FEC2C7
:101099007F113B22E5EF20E6037520000520903FF4
:1010A900FFE520146006901DFF146000930460039F
:1010B90075EF1253D9BF7581C043FF8012059E7524
:1010C900EF0243B203E5B3240420E70DF521E5E37C
:1010D90020E0068521B343E301120F397580FF75BE
:1010E900A40075F1D475D4EF75908775A54075F294
:1010F900FF75D5BF75A60175E24275DB4675EA0233
:10110900E4F8F6D8FD756B01120F4E1215CF7898D9
:101119008676753001C2AF1205B71205C71205AD43
:101129001205CE1205AD1205D51205ADC2AF78FA7A
:1011390079FA308407D9FBD8F7021C00120FB712CD
:101149000FF0113A113B78988676120F397588504D
:1011590075891275C82475910475D84075A82275CA
:10116900B80275E690759B80759D0075D10E75BCAA
:101179005875BB0375BA1175E88012059ED2AF1276
:1011890008AB53DACF207E0343DA20307E0343DAFB
:101199001043DA01C2D8C2711205B7D2617B037A52
:1011A9000CE55E70077A0CDB030211351205AD20E0
:1011B9007003021135C270E55FC3940240E1E52F67
:1011C900541F856160F561B560D5DAD5C26153DA1E
:1011D900CF207E0343DA20307E0343DA10C2D8C21F
:1011E9007178A2E67008D274E52F54E0F52FC27524
:1011F9007529001205B2307409C3E529940A400221
:10120900D2751205A378023074027800C3E55F989D
:1012190040F0C2AF1205C71205C71205C7D2AF12F7
:1012290005B7754D007888E6B40302610C1205A371
:10123900788CE6C39401500302130CE530C3940182
:10124900500302130C207435C3E55F94FF50030269
:10125900130CC2AF1205DCD2AF1205B2C3E55F941D
:101269000150EFC2AF1205C71205A81205C7D2AFC8
:101279001205B2C3E55F94FF40E90217777F02D2F6
:101289007F113B1205B2C2AFC27F113BAE5FC3E50E
:101299005F947FD2AF407612059EC2AF1205DCD2B1
:1012A900AFDFDC1172C3EE94057897F61205B71219
:1012B90016111216FA7F0AD27F113B1205B2C2AF7C
:1012C900C27F113BAE5FC3E55F947FD2AF50E61298
:1012D900059EC2AF1205C71205A81205C7D2AFDF16
:1012E900D61172EE24057896F61205B71216111268
:1012F90017291205B2113BC3E55F94FF5002414E15
:10130900021777C3E55F954D4003855F4D1205B21E
:1013190078017988E7B403027805C3E55F9840024C
:10132900412EC2AF1205DC1205DC1205DCD2AF1268
:1013390005B7753000E4F531F5320531E531F47062
:10134900390532789AE67819146012783214600DEA
:10135900787D14600878FA146003753200C3E532A9
:1013690098401715327531B478998676C2AF12054F
:10137900DCD2AF789886761205B21205A8E52A70F4
:1013890005307402213578012074027806C3E55FBF
:101399009840A77888E6C3940360031205B2E52A4A
:1013A9007003021135C2AF120F39E4F522F523F5A6
:1013B90024F525F526F56AD2AF7885E6C333F568B5
:1013C900E4F545F546F547F548F549F573F52CF586
:1013D9002DF53775730875BB1012059E1208AFE518
:1013E900E820ECFBA8BDA9BEE97001F888741208D1
:1013F900B375730875BB107887E6FE7602120FB7CE
:101409007887EEF6C2AF7564FF12094B85226485B1
:101419002265852266D2AF752201752401752501E1
:1014290075260185636C756D017888E6B40307C27A
:101439007D307602D27DD268D269753300120E9B57
:10144900120EC212096B12097212096B1209721279
:10145900096B02146BC2AF120FB7D2AF7573007567
:0E146900BB03120BF61206A7120D11120D5B3B
:10147700120972120BE5306D03120703206703127E
:10148700084E306703120895120D11120D821209CA
:1014970072120BF6306D03120738120D11120DFB85
:1014A700120972120BE5306D03120796120D111215
:1014B7000E22120972120BF6306D031207F3120D8A
:1014C70011120E9B1209721208AF120BE5120D11C1
:1014D700120EC21208B3120972306935206B3285B9
:1014E700676485676585636C756D0179187A0CC3C8
:1014F700E53399400FC269D26A8A35856764856783
:1015070066021518C3E55F9401400302146B0215C8
:1015170095306A1B206B18E535147004C26A815E2A
:10152700F535C3E55F9401400302146B0215957509
:101537003600C3E56278FA985054307404E52A609F
:101547004D7888E6B40317207D05207607A165301E
:101557007602A165206B07D26B85676481AA78F054
:10156700306B058567647820C3E541985002816B2D
:10157700306B1BC26BC27D307602D27DD26A753565
:1015870012856764816B0536E55F6002A198753641
:1015970000C2AF120F397887E6FE7602120FB778CE
:1015A70087EEF6E4F522F523F524F525F526F5680B
:1015B700C268D2AF12059E120F39307409C3E536DF
:1015C700940540022135613E901A0D78201216537A
:1015D700E520B4550CA3121653E520B4AA0302154F
:1015E700F1120F4E121611021610901A0378807B13
:1015F7000A121653A308DBF9901A0F788C7B18127E
:101607001653A308DBF9901A2722C2AF12169212BB
:10161700166C901A00740E121658A37404121658FA
:10162700A37414121658901A0378807B0A1216575F
:10163700A308DBF9901A0F788C7B18121657A308AA
:10164700DBF91216A5121683901A2722E493F622C5
:10165700E6438F01538FFD75EF0275B7A575B7F197
:10166700F0538FFE22438F02438F0175EF0275B748
:10167700A575B7F1901A0DF0538FFC22901A0D74CF
:1016870055D158901A0E74AAD158227A3079D07849
:1016970020901A40D153E520F709A3DAF7227A30D0
:1016A70079D0901A40E7D15809A3DAF922AB77A885
:1016B70078BB01027980BB02027981BB0302798280
:1016C700BB04027984BB05027986BB06027992BB0B
:1016D70007027987BB080279A3BB0902799CBB0A79
:1016E700027988BB0B027989E8F7227C051205B7D6
:1016F700DCFB22C2AF1205C71205CE1205D51205B3
:10170700DC1205A81205C71205CE1205D51205DC95
:101717001205A81205C71205CE1205D51205DCD28F
:10172700AF22C2AF1205DC1205D51205CE1205C7CE
:101737001205A81205DC1205D51205CE1205C7122F
:1017470005A81205DC1205D51205CE1205C7D2AFC2
:1017570022AE77AF78C2AF1205C71205C71205C709
:101767001205A8DEF21205DC1205A8DFF8D2AF22B7
:10177700D1FAD1F2D1F2757701757801757900F157
:10178700587C05AD5F1205B7C3ED955F70F5C3E5EE
:101797005F9401400AC3E55F94FF40320217B3D15B
:1017A700B4D111D1FAC2AF75EF12D1F2DCD50579F8
:1017B700C3E5799403500280C6D1F20578E5771422
:1017C70090009F93F808C3E57898500280AED1F255
:1017D700D1F20577C3E577940C5002809C120F4E27
:0917E700D111C2AF75EF12D1F26D
:0319FD0002109D38
:101A00000E0414090904FF03FF0A03010155AA018A
:101A1000FFFFFFFFFF03FFFFFF25D0285004FF0259
:081A2000007AFF01010003FF41
:101A400023484B696E67323041232020202020201C
:101A500023424C48454C4923463333302320202031
:101A60002020202020202020202020202020202076
:101C0000C2AFC2D353D9BF7581C043B20343FF8073
:101C1000752438752503B1C975EF0275E24043F1AB
:101C20001053A4EF75D400D2847DFA780379E67C52
:101C300010752200752300901DD67B0675249875BB
:101C400025013084028142208408D8FBD9F9DCF7D1
:101C500081B4308408D8FBD9F9DCF781B4B189E4C8
:101C600093A3C39A6004DDC381B4DBDBB17B600264
:101C7000812B7B08E493FAA3B15CDBF87A30B15C8A
:101C8000752200752300B17BEAFCEBFDC3ED94FEE9
:101C9000400EB17B8A278B28ED30E0048A828B834B
:101CA000B17B7AC270D8C3ED94FE601350CEBD00F4
:101CB00025EC60097520007521FF0200008100A855
:101CC00027A9280809D804D90281D3B17FEA89AAB3
:101CD000F281C50D81A0C3ED94035049EDA2E092BD
:101CE000007AC5C3E5829400E583941C50902000DF
:101CF00010438F02438F0175B7A575B7F1F030001F
:101D00001FA827A9280809438F01538FFDD804D99C
:101D100002A12089AAE275B7A575B7F1F0A3A10DBC
:101D2000538FFC817C7AC1BD030CE493A3FAB140CC
:101D3000DCF8B138817C817EAA22AB23B15CEBFA5E
:101D4000EA6222752608C3E52313F523E52213F57D
:101D50002250066323A0632201D526EAB1C9B1C986
:101D600075260AEAF4200102D284300102C284B14D
:101D7000C9C3134002C201D526EB22B17FEAFB2082
:101D80008402A17F308402A184752608AE24AF2589
:101D9000C3EF13FFEE13FEB1CDB1C9C3EA13308414
:101DA000024480FA30E703632201C3E52313F523DD
:101DB000E52213F52250066323A0632201D526D91C
:101DC000E52265236523F52222AE24AF250E0FDE22
:101DD000FEDFFCD20122424C48656C693437316326
:041DE000F3300601D5
:00000001FF
